:0300000002116981
:03000B000200A54B
:03002B000202DEF0
:03005B0002046735
:030073000204364E
:1000800002030406080C10182030406080040608A3
:100090000C10182030406080A0C00D0D0405060D26
:1000A0000503030302306306C26385768A32C2AF5A
:1000B000C0D0C0E020620C20680241BD3066024121
:1000C0007DE473C3E525334009758A00D263F57674
:1000D00001D4F58AC262E525F47002214420680249
:1000E000212B207213758B00758D00D0E0D0D0C20B
:1000F00092C296C294D2AF32C292C296C294741681
:10010000D5E0FDE53C1420E21520E10D207D02D272
:1001100097307D02D29302013ED29502013E207DAE
:1001200002D293307D02D29702013E758B00758D0D
:1001300000D0E0D0D0C292C296C294D2AF32758BBA
:1001400000758D00D0E0D0D0D2AF3241BDE5256042
:100150000A207D02D292307D02D296C29441BDE542
:10016000256002D294207D02C296307D02C2924167
:10017000BDE525600A207D02D296307D02D2922014
:100180007D02C292307D02C29641BD207D02C293A3
:10019000307D02C297207D02C297307D02C29374E7
:1001A0001AD5E0FDE525600A207D02D292307D025D
:1001B000D296C29441BD207D02C293307D02C29787
:1001C000C295741AD5E0FDE525600A207D02D29221
:1001D000307D02D296C29441BDC295207D02C29369
:1001E000307D02C297741AD5E0FDE5256002D294F5
:1001F000207D02C296307D02C29241BDC295207D13
:1002000002C297307D02C293741AD5E0FDE52560E5
:1002100002D294207D02C296307D02C29241BD205E
:100220007D02C297307D02C293C295741AD5E0FD5B
:10023000E525600A207D02D296307D02D292207D93
:1002400002C292307D02C29641BD207D02C297302B
:100250007D02C293207D02C293307D02C297741A40
:10026000D5E0FDE525600A207D02D296307D02D2E0
:1002700092207D02C292307D02C29641BD30723D15
:10028000E53C20E21A20E129207D02C293307D0264
:10029000C297207D02C297307D02C2930202BD2028
:1002A000E1E6207D02C293307D02C297C295020230
:1002B000BDC295207D02C297307D02C293E525F430
:1002C000C3334009758A00D263F57641CFF58A754C
:1002D0008B00758D00D262D0E0D0D0D2AF32C2AFE9
:1002E000C2AD53E6EFC0D0C0E0D2D3D2AFE5776065
:1002F00009E574600575740061E1757401C2CEE5AD
:100300002960072074461529614C78007900E58042
:10031000307E01F430E50278FF53DACF207E0343CC
:10032000DA20307E0343DA10C2D8C271E580307E15
:1003300001F430E50279FFC3E89970CE30610375AE
:1003400029182074037529188859D270E52A600489
:10035000152A615C20740543DA01C2D8207002615D
:10036000C3A859206102C2702074367982B7043163
:10037000C3E894F0400374F0F8E8C4540F28F87907
:1003800084B7030261A1C313C3138721200802C3EA
:1003900013200A06C3C898F861A128F8500374FF17
:1003A000F88822306915E5222408F52250037522C9
:1003B000FFC3E522955E4003855E227882B604186D
:1003C000852224A824C3E524955E4002A85EC3E8E4
:1003D00095604002A8608825C3E52594404002D27C
:1003E0006420CF0CD0E0D0D0C2D343E610D2AD32DF
:1003F000E5776009E5756005757500812A757501F9
:10040000C2CF7801E52960053074021529C3E5598A
:1004100094014005755C00812A755D00756400E5F6
:100420005C2401F55C5003755CFFD0E0D0D0C2D3F2
:1004300043E610D2AD32C0D0C0E0C2AF53917F537B
:10044000E67FC260C3E55033F550E55133F5517591
:100450009100C3E49550F594E49551F59575910498
:10046000D0E0D0D0D2AF32C2AF53E6EFC2ADC0D0F1
:0E047000C0E0C0F0D2D3D2AFA8FBA9FCE57764
:10047E006007C3E913F9E813F8C2D830710281D9C5
:10048E0053DACF207E0343DA10307E0343DA20D2D4
:10049E0071E580307E01F420E50281B0882689273F
:1004AE00E11553DACF207E0343DA20307E0343DAA0
:1004BE0010C2D8C271307402E1017800E580307E3E
:1004CE0001F430E502E1018859C1E853DACF207E0C
:1004DE000343DA20307E0343DA10C271206102A199
:1004EE00A953DACF207E0343DA10307E0343DA209D
:1004FE00C2D8D27188548955C3E89552F8E99553FC
:10050E00F9E4FB7E027A00C3E8948CE9940050056E
:10051E00755800A199C3E894C8E994005008E4D234
:10052E00E4FB7A0AA176C3E89468E994015008E4E2
:10053E00D2E3FB7A0FA176C3E894D0E99402500877
:10054E00E4D2E2FB7A1EA176C3E894A0E9940550AA
:10055E0008E4D2E1FB7A3CA176C3E89498E99408CA
:10056E005008E4D2E0FB7A787E00C3E89556FCE9A9
:10057E009557FD30E708ECF42401FCEDF4FD7558B9
:10058E0000C3EC9AED9E500375580188568957A802
:10059E0054A955885289537802C1E8C3E89526F8C4
:1005AE00E99527F9307C02C1CC307B02C1CC307A80
:1005BE0002C1C5207502A1CCE9FDE8FCA1EBE9C39F
:1005CE0013F9E813F8307902C1C5E9C313F9E8133A
:1005DE00F8307802C1C5E9C313FDE813FC2061268B
:1005EE00C3EC941CED94024002C102ED7018C3ECF2
:1005FE0094C850120528C3E528940A5002E10175EB
:10060E005900D270E101E528600215287400207FA0
:10061E000B7888E67896B40302789EE624FAFEE418
:10062E003400FFC3EC9EFCED9FFD92087888E6B483
:10063E000327A2085009207D20C2AFD27DC15430BD
:10064E007D17C2AFC27DC292C296C294C293C297A8
:10065E00C295206902D26BD2AFA2085017E6B4033E
:10066E000DECF42401FCEDF43400FD02068278005A
:10067E007900C1CC7888E6B40315EC33FCED33FD7C
:10068E00C3EC940AFCED9400FD50047C007D00C385
:10069E00EC94FFED9400400678FF7900C1CCEC8518
:1006AE006FF0A4C5F0A2F733F8790040030206E814
:1006BE0078FF79000206E8E9C313F9E813F8307CF5
:1006CE000EE9600278FFC3E81338F8E43400F9C38A
:1006DE00E894FFE99400400278FF8859D2702061B7
:1006EE0002E101741FF4552F4BF52FC274E42B70E9
:1006FE0002D27475291830740375290A306102E12B
:10070E001520740353DAFE752A06307403752A0A0F
:10071E00D0F0D0E0D0D0C2D3D2AD43E610327901C2
:10072E0002074A790302074A790A02074A791E022A
:10073E00074A796402074A79C802074A7817E4D54E
:10074E00E0FDD8FAD9F6227A147B780207717A1076
:10075E007B8C0207717A0D7BB40207717A0B7BC812
:10076E00020771AC257525017902B27DE4C295D5DB
:10077E00E0FDE5256002D294D5E0FDC294D5E0FD02
:10078E00D295D5E0FDE525600A207D02D292307D1E
:10079E0002D296E570D5E0FD207D02C292307D0238
:1007AE00C2967496D5E0FDD9C1EAF8D5E0FDD8FB26
:1007BE00DBB1C2958C2522C37C007D0075F000054F
:1007CE00F0EA33FAEB33FB50F6EB13FBEA13FAC302
:1007DE00E9FFE8FEE89AF8E99BF95004EFF9EEF824
:1007EE00B3EC33FCED33FDD5F0DFEDF9ECF822E898
:1007FE0089F08A20D2D4F8A9F07B0030F70B7BFF6A
:10080E00F42401F8E9F43400F9E88520F0A4ADF001
:10081E00F8E98520F0A4AFF0FEED2EF974003FFA52
:10082E007C04C3EA13FAE913F9E813F8DCF48BF04D
:10083E0030F70AE8F42401F8E9F43400F9E889F015
:10084E00C2D4F8A9F0227882B604030208B1C3E537
:10085E005994014003020879852224E4F53EF53FC0
:0F086E00F540F541F542F5470208B17882E6FC06
:10087D00754701E522F523783879C7AA3AAB3BC312
:10088D00EB13FBEA13FAEC146013C3EB13FBEA133F
:10089D00FAEC14146007C3EB13FBEA13FA1207C545
:1008AD00883E893F22E5476034C3E53E9523F8E550
:1008BD003F9400F9500CC3E89480E994FF40160270
:1008CD0008E6C3E8947FE9940050030208E6787FB8
:1008DD0079000208E6788079FF8843894422E5474C
:1008ED006058E5432540F8E5443541F9854420E459
:1008FD00300701F43542FA30E709C3EA94F04015A8
:10090D00020928C3EA940F500302092878FF79FFE2
:10091D007A0F020928780079007AF0C3E524955EF4
:10092D005006E52460092141E54420E70D2141E50C
:10093D004430E706884089418A4222E54770030228
:10094D0009AC78A1E6FAC3E54333F8E54433F9126F
:10095D0007FDE930E70BC3E89480E994FF401321CC
:10096D0083C3E8947FE9940050022183787F790056
:10097D002183788079FFE820E715C3E52398F840B7
:10098D0009C3E8940140030209AA78010209AAE803
:10099D00F424012523F840030209AA78FF88452293
:1009AD00E5477003020A0F78A2E6FAA841A94212A0
:1009BD0007FDE930E70CC3E89401E994FF40160206
:1009CD0009E6C3E894FFE9940050030209E678FFB5
:1009DD0079000209E6780179FFE920E715C3E545BD
:1009ED0098F84009C3E894014003020A0D7800020B
:1009FD000A0DE8F424012545F84003020A0D78FF9D
:100A0D0088242278FFC264E52D5406702FD264C36A
:100A1D00E53B940A4009C3E52594405002C264E5C4
:100A2D003B601974FF853BF0848537F0A4F8C5F061
:100A3D00600278FFC3E895615002A8618860227852
:100A4D0083E6F520120F8C75E89012072C75E8904F
:100A5D00E5E820ECFBA8BDA9BE121022756B01754F
:100A6D006C00C3740013FD740113FC74012CFC7431
:100A7D00003DFDECFAEDFBC3E89AE99B4014E56BF4
:100A8D002401F56BE56C3400F56CEA2CFAEB3DFBBB
:100A9D0080E5AE6BAF6CC3E56C13F9E56B13F8C372
:100AAD00E913F9E813F8E56B28F569E56C39F56A92
:100ABD007A03C3E913F9E813F8DAF7AA201A7009D3
:100ACD00756B00756C00020AE61AEA6008EE28FEE6
:100ADD00EF39FFDAF88E6B8F6C2275E890227883F0
:100AED00E6FFE5E820ECF7A8BDA9BE056DC3E56DF1
:100AFD0094084052756D00E9FA79A0E76044EA70F8
:100B0D0007E56E601B020B21C3E8956E6010E56E64
:100B1D005006600C14020B2D0460F9020B2DE56ECE
:100B2D00F56EC39472401B755EC0C394044013757B
:100B3D005E80C39404400B755E40C39404400375FE
:100B4D005E0075BB0822EFC39401601BC3E894FFE0
:100B5D00E994035012C3E8956BE9956C5009E55E75
:100B6D00601A155E020B89E55EF46010055E7888EB
:100B7D00E6B40308E55E24044002F55EA85EC3E515
:100B8D0024985002A824C3E8955F400AA85FE55F4A
:100B9D00F46003855F5E7982B7040261B4C3E895A2
:100BAD00604002A8608825E56DB4070375BB10226F
:100BBD00743279A387F0A4C5F0A2F733F8C3E89592
:100BCD005E4002A85E882288248825886122753AB5
:100BDD0000753B7F2275C820A8CCA9CD75C824C34C
:100BED00E913F9E813F8AA38AB3988388939C3E81D
:100BFD009AF8E99B547FF9AA3AAB3BAC3AAD3B7EF0
:100C0D00047F02C3EB940440021E1FC3EB94084003
:100C1D00021E1FC3ED13FDEC13FCDEF7C3EA9CFAB5
:100C2D00EB9DFBEF6009C3E913F9E813F8DFF7EA71
:100C3D0028FAEB39FB8A3A8B3B400122753AFF7556
:100C4D003BFF223060028150854C50854D51D26062
:100C5D0043E680227892E6FFC3E535948240010F8A
:0E0C6D00C3E53594A040010FC3EF940640028A
:100C7B007F057E021E3072010EC3E53B94035006C6
:100C8B000E0E3072010EC3E53B940250060E0E3071
:100C9B0072010EA93BA83A7A04C3E913F9E813F8D9
:100CAB00DAF7C3E89EF8E99400F94009C3E8940227
:100CBB00E9940050047802E4F9E9FBE8FAC3E9137C
:100CCB00FDE813FC884C894DC3EF94036037EF208C
:100CDB00E00DE82CF8E93DF9ECFAEDFB020CFDE830
:100CEB0028F8E939F9C3E89402F8E99400F97A0293
:100CFB00E4FBC3EF9403400D8A4E8B4F8848894920
:100D0B008C4A8D4B22884E894F8A488B498C4A8D51
:100D1B004B22306002A11DD26043E680E52D5406C4
:100D2B00602EA83AA93BE53494085006E820E0026F
:100D3B00A94DC3E833F8E933F9759100C3E498F58D
:100D4B0094E499F595759104D26053917F43E680B5
:100D5B0022D265753D00752000020D6FD265753D81
:100D6B0000752040E52D54066002C265D2AF2060AD
:100D7B0005E53D60012278017A02C3E53B9405400D
:100D8B00027802C3E53B940A40027803C3E53B9427
:100D9B000F40027A03306904781E7A01206007E560
:100DAB003D6003D2AF22D2AF0000C2AFC3E53BFB25
:100DBB00940F40027B0FEB0430730123206201235D
:100DCB00F93069027982E58D13E58B13C39940CC19
:100DDB00053DEAFBE59BF45440B52004DBF6C11658
:100DEB00206502A16FC265759100AE3AAF3BC3EEB1
:100DFB0033FEEF33FFC3E49EF594E49FF5957591B5
:100E0B0004D26053917F43E680A16F306502A16FDE
:100E1B00D88AD2AF2230690B0534206016753400A6
:100E2B00020E3E20600D20650A206B07158115818F
:100E3B0002163122A84EA94FC3E833F8E933F975EE
:100E4B00910053917FC3E498F594E499F5957591CE
:100E5B0004854850854951D26043E68022780030A2
:100E6B0064053065027801E53575F007A4F9E5F006
:100E7B0028F5F0E9A2F013A2F113A2F213F535C392
:100E8B0094785003753578C3E53595364008D266AE
:100E9B00C292C296C294306002C1A1854A50854B62
:100EAB0051D26043E68022C2AFC293C297C2953043
:100EBB00720B90021F741AD5E0FD020EC8207D0242
:100ECB00D293307D02D297759F40753C020210077A
:100EDB00C2AF207D02C296307D02C2923072179053
:100EEB0001FCC295207D02C297307D02C293741A19
:100EFB00D5E0FD020F0490015F306206E52560022C
:100F0B00D294207D03759F41307D03759F43753CC3
:100F1B0003021007C2AFC293C297C29530720B90F7
:100F2B0001D9741AD5E0FD020F35207D02D297301E
:100F3B007D02D293207D03759F43307D03759F41C6
:100F4B00753C04021007C2AFC2943072179001B601
:100F5B00207D02C293307D02C297C295741AD5E0F0
:100F6B00FD020F7290014D30620EE525600A207D67
:100F7B0002D292307D02D296759F40753C050210CD
:100F8B0007C2AFC293C297C29530720B90018B749C
:100F9B001AD5E0FD020FA2D295207D03759F41303B
:100FAB007D03759F43753C06021007C2AF207D027F
:100FBB00C292307D02C29630721F90024A207D028F
:100FCB00C293307D02C297207D02C297307D02C250
:100FDB0093741AD5E0FD020FE790017130620EE5B4
:100FEB0025600A207D02D296307D02D292207D03AD
:100FFB00759F43307D03759F41753C01306B131218
:10100B001022741AD5E0FD7416D5E0FDD293D29759
:10101B00D295C266D2AF2290014BC292C296C294B5
:10102B00C293C297C295C26222788076090876096C
:10103B000876040876010876030876FF08760A0816
:10104B007601087601087601788C76010876FF0820
:10105B0076FF0876FF0876FF0876FF08760308769A
:0E106B00FF0876FF0876FF0876250876D00885
:1010790076280876500876040876FF0876020876FE
:101089000008767A0876FF087601227887E6FFC29B
:1010990072BF0302D2727888E6C394036008C27DE6
:1010A900E630E102D27DC27E7889E630E102D27E65
:1010B900C3EF94026008758E01D2730210CC758E4D
:1010C90000C273227880E6149000809378A1F678A4
:1010D90081E6149000809378A2F61122227886E6A0
:1010E9001490008D9378A3F611222222789CE6753C
:1010F90036FF75370CB402067536A075370AB40386
:101109000675368275370522227896E6FA7897E6CB
:10111900FB307F047A007BFFC3EB9AFCC3948250B7
:10112900027C82756F00056FEC856FF0A4C3E5F052
:10113900948040F222D27F311212073B7A007B0061
:101149007C10120731E5592AFA74003BFBDCF37C69
:1011590004C3EB13FBEA13FADCF7FEC27F31122258
:10116900E5EF20E6037520000520903FFFE52014F8
:101179006006901FFF1460009304600375EF12C2AC
:10118900D353D9BF7581C043FF8012072C75EF0275
:1011990043B203E5B3240420E702F5B311227580B5
:1011A900FF75A40075F13075D4DF75900375A5FC42
:1011B90075F2FC75D50175A60175E2411134121657
:1011C9006978988670C2AF12074512075512073B16
:1011D90012075C12073B12076312073BC2AFE4F820
:1011E900F6D8FD78C879C8308507D9FBD8F7021C2D
:1011F900001134121669119411CD11E611F411F58B
:101209003111311278988670112275B68075A9004E
:1012190075770075885075891275C824759104759C
:10122900D84075A82275B80275E690759B80759DA2
:101239000075D10E75BCC075BB0875BA1175E8800B
:1012490012072CD2AF120A4C43DA01C2D8C271126A
:101259000745753001D2617B037A0CE55870067A2F
:101269000CDB0221E512073B20700221E5C270E583
:1012790059C3940240E3E52F541F855B5AF55BB5CA
:101289005AD7DAD7C26153DACF207E0343DA203046
:101299007E0343DA10C2D8C271C2757528001207DD
:1012A90040307409C3E528940A4002D27512073107
:1012B90078023074027800C3E5599840F0C2AF1241
:1012C9000755120755120755D2AF12074575460043
:1012D9007888E6B4030261B5120731788CE6C394C5
:1012E9000150030213B5E530C3940150030213B54D
:1012F900207435C3E55994FF50030213B5C2AF12E8
:10130900076AD2AF120740C3E559940150EFC2AF43
:10131900120755120736120755D2AF120740C3E517
:101329005994FF40E90218107F02D27F3112120747
:1013390040C2AFC27F3112AE59C3E559947FD2AFD3
:10134900407412072CC2AF12076AD2AFDFDC313EFC
:10135900C3EE94057897F61207451216AA12179349
:101369007F0AD27F3112120740C2AFC27F3112AE5B
:1013790059C3E559947FD2AF50E612072CC2AF1278
:101389000755120736120755D2AFDFD6313EEE2484
:10139900057896F61207451216AA1217C2120740C7
:1013A9003112C3E55994FF40F4021810C3E5599569
:1013B90046400385594612074078017988E7B40306
:1013C900027805C3E55998400241D9C2AF12076AAC
:1013D90012076A12076AD2AF120745753000E4F5A1
:1013E90031F5320531E531F470390532789AE6780C
:1013F90019146012783214600D787D14600878FA37
:10140900146003753200C3E53298401715327531FF
:10141900B478998670C2AF12076AD2AF789886708D
:10142900120740120736E529700530740221E57864
:10143900012074027806C3E5599840A77888E6C365
:1014490094036003120740E529700221E5C2AF1138
:1014590022E4F522F523F524F525D2AF78858662B5
:0E146900F53EF53FF540F541F542F56DF547CE
:10147700F52CF52DF535120BDB756D0875BB1012C4
:10148700072C120AE7E5E820ECFBA8BDA9BEE97026
:1014970001F8886E120AEB756D0875BB107887E640
:1014A700FE760211947887EEF6C2AF755EFF120BD7
:1014B700BD85225E85225F852260D2AF75220175C8
:1014C7002401752501855D6475650175B69075A95B
:1014D70003757701D268D269753400120F8C120F29
:1014E700B6120BDB120BE2120C610214FE11221171
:1014F70094756D0075BB08120D67120E20120E3F12
:10150700120854120E68120EB2120BE2120C50128D
:101517000C61120D1D120D5C120E20120E3F1208E7
:10152700B2120A10120E68120EDB120BE2120C50E6
:10153700120C61120D1D120D67120E20120E3F12B2
:1015470008EB120E68120F1F120BE2120C50120C4E
:1015570061120D1D120D5C120E20120E3F1209486A
:10156700120E68120F51120BE2120C50120C61127C
:101577000D1D120D67120E20120E3F1209AD120E2D
:1015870068120F8C120BE2120C50120C61120D1D17
:10159700120D5C120AE7120E20120E3F120AEB120E
:1015A7000E68120FB6120BE2120C50120C61120DDC
:1015B7001D306938206B3585615E85615F855D64A7
:1015C70075650179327A0AC3E534994012C269D246
:1015D7006A8A3385615E755FFF7560200215F3C304
:1015E700E559940140030214FE021631306A1E20A9
:1015F7006B1BE533147007C26A755EFF81F4F53320
:10160700C3E559940140030214FE021631C3E55C99
:1016170094FA5016307404E529600FC3E53B78F05F
:10162700306B02786098500281FEC2AF1122788732
:10163700E6FE760211947887EEF6E4F522F523F5B7
:1016470024F525F562C26875B68075A9007577001F
:10165700D2AF12072C1122307406E529700221E55A
:1016670061E7901A0D78201216ECE520B4550CA30B
:101677001216ECE520B4AA0302168A11341216AA30
:101687000216A9901A0378807B0A1216ECA308DBCE
:10169700F9901A0F788C7B151216ECA308DBF990DA
:1016A7001A2422C2AF12172B121705901A00740DB5
:1016B7001216F1A374021216F1A374131216F19005
:1016C7001A0378807B0A1216F0A308DBF9901A0F29
:1016D700788C7B151216F0A308DBF912173E121748
:1016E7001C901A2422E493F622E6438F01538FFDC0
:1016F70075EF0275B7A575B7F1F0538FFE22438FCB
:1017070002438F0175EF0275B7A575B7F1901A0DF2
:10171700F0538FFC22901A0D7455D1F1901A0E7464
:10172700AAD1F1227A3079D07820901A40D1ECE50D
:1017370020F709A3DAF7227A3079D0901A40E7D157
:10174700F109A3DAF922AB71A872BB01027980BB58
:1017570002027981BB03027982BB04027984BB054B
:10176700027983BB06027986BB07027992BB08021E
:101777007987BB0902799CBB0A027988BB0B02797E
:1017870089E8F7227C05120745DCFB22C2AF120766
:101797005512075C12076312076A120736120755BC
:1017A70012075C12076312076A12073612075512EF
:1017B700075C12076312076AD2AF22C2AF12076A29
:1017C70012076312075C12075512073612076A12CF
:1017D700076312075C12075512073612076A1207CA
:1017E7006312075C120755D2AF22AE71AF72C2AF58
:1017F700120755120755120755120736DEF2120760
:101807006A120736DFF8D2AF2212179312178B121C
:10181700178B7571017572017573001217F17C05CD
:10182700AD59120745C3ED955970F5C3E5599401B4
:10183700400AC3E55994FF403702185412174D1256
:1018470016AA121793C2AF75EF1212178BDCD105C8
:1018570073C3E5739403500280C112178B0572E5B9
:0E186700711490009A93F808C3E5729850022D
:1018750080A812178B12178B0571C3E571940C5054
:101885000280941210341216AAC2AF75EF12121705
:011895008BC7
:101A00000D02130909040103FF0A01010155AA018E
:101A1000FFFFFFFFFF03FFFFFF25D0285004FF0259
:051A2000007AFF01FF48
:101A40002358526F746F723230412320202020209F
:101A500023424C48454C492346333930232020202B
:101A60002020202020202020202020202020202076
:101C0000C2AFC2D353D9BF7581C043B20343FF8073
:101C1000752438752503B1BF75EF0275E24043F1B5
:101C20002053A4DFD285780379E67C1075220075F5
:101C30002300901DCC7B0675249875250130850204
:101C4000813D208508D8FBD9F9DCF781AD308508C6
:101C5000D8FBD9F9DCF781ADB17FE493A3C39A60D7
:101C6000028126DBDDB171600281267B08E493FAF4
:101C7000A3B152DBF87A30B152752200752300B15E
:101C800071EAFCEBFDC3ED94FE400EB1718A278B27
:101C900028ED30E0048A828B83B1717AC270D8C398
:101CA000ED94FE601050CEBD0022EC600675200061
:101CB0000200008100A827A9280809D804D90281B8
:101CC000C9B175EA89AAF281BB0D8199C3ED94036C
:101CD0005049EDA2E092007AC5C3E5829400E58305
:101CE000941C5093200010438F02438F0175B7A5B9
:101CF00075B7F1F030001FA827A9280809438F0104
:101D0000538FFDD804D902A11689AAE275B7A5752B
:101D1000B7F1F0A3A103538FFC81757AC1BD030C09
:101D2000E493A3FAB136DCF8B12E81758177AA224B
:101D3000AB23B152EBFAEA6222752608C3E52313FE
:101D4000F523E52213F52250066323A0632201D573
:101D500026EAB1BFB1BF75260AEAF4200102D28596
:101D6000300102C285B1BFC3134002C201D526EBC8
:101D700022B175EAFB208502A175308502A17A7532
:101D80002608AE24AF25C3EF13FFEE13FEB1C3B197
:101D9000BFC3EA133085024480FA30E703632201AF
:101DA000C3E52313F523E52213F52250066323A090
:101DB000632201D526D9E52265236523F52222AECB
:101DC00024AF250E0FDEFEDFFCD20122424C486517
:0A1DD0006C6934373132F3900601DC
:00000001FF
